:0300000002304586
:0C30450078FFE4F6D8FD75814A02308C5B
:100E9E000A53746172743A20004950436F6E6E6546
:100EAE0063745245510A004950436F6E6E65637408
:100EBE00003E432C562C43432CC0E4E0EFF2E5F009
:100ECE0020D1E8EDEAEEEC49500A003E432C4D41AC
:100EDE00432C25303262583A25303262583A25304A
:100EEE003262583A25303262583A25303262583AD8
:100EFE0025303262582C4D414320E0E4F0E5F10AF2
:100F0E00003E432C5645522C20332E3120EEF2203B
:100F1E0025732025732CC2E5F0F1E8FF20495020FF
:100F2E00ECEEE4F3EBFF0A004E6F76203033203206
:100F3E003030370030383A35313A3533003E432CB5
:100F4E004C442C50524F473A202020202020202065
:100F5E002020202020202020202020202020202083
:100F6E002020202020202020202020202020202073
:100F7E002020202020202020202020202020202063
:100F8E00202020202020202020202020202CC4E0E3
:100F9E00F2E020EFF0EEF8E8E2EAE828F4E0E9EB20
:100FAE00290A003E2A2C312CCEF1EDEEE2EDFBE5C6
:100FBE0020EFE0F0E0ECE5F2F0FB20F1E5F2E5E207
:100FCE00EEE3EE20E8EDF2E5F0F4E5E9F1E00A00FB
:100FDE003E412C4130312C2562752E2562752E2511
:100FEE0062752E2562752C495020E0E4F0E5F12063
:100FFE00E0E4E0EFF2E5F0E00A003E412C41303251
:10100E002C2562752E2562752E2562752E2562752C
:10101E002C495020E0E4F0E5F120EEF1ED2E20F128
:10102E00E5F0E2E5F0E00A003E412C4130332C259C
:10103E0062752E2562752E2562752E2562752C49D8
:10104E005020E0E4F0E5F120F0E5E72E20F1E5F0A8
:10105E00E2E5F0E00A003E412C4130342C25627569
:10106E002E2562752E2562752E2562752CCCE0F12B
:10107E00EAE020F1E5F2E80A003E412C4130352C41
:10108E002562752E2562752E2562752E2562752CAC
:10109E00D8EBFEE70A003E532C4130362C25627504
:1010AE002CC2F0E5ECFF20EEE6E8E42E20EAE2E8C2
:1010BE00F2E0EDF6E8E820282A3130ECF1290A00BA
:1010CE003E2A2C312CC4EEEF2E20EFE0F0E0ECE5C2
:1010DE00F2F0FB20F1E5F2E5E2EEE3EE20E8EDF2D0
:1010EE00E5F0F4E5E9F1E00A003E422C5330312CF4
:1010FE002562752CC6E4E0F2FC20E7E0EFF0EEF19D
:10110E00E020F1EEE5E4E8EDE5EDE8FF20EEF2207B
:10111E00F1E5F0E2E5F0E00A003E422C5330322CCD
:10112E002562752CCEE1ECE5ED20F120F1E5F0E243
:10113E00E5F0EEEC20E1E5E720EAE2E8F2E0EDF69C
:10114E00E8E90A003E422C5330332C2562752CCF31
:10115E00E5F0E5E7E0EFF3F1EA20EFF0E820EFEE5F
:10116E00F2E5F0E520F1E2FFE7E820F120F1E5F00D
:10117E00E2E5F0EEEC0A003E422C5330342C2562B0
:10118E00752CCDE5F220EFE5F0E5E4E0F7E820E49C
:10119E00E8E0E3EDEEF1F2E8EAE820E220F1E5F036
:1011AE00E2E5F00A003E422C5330352C2562752CB8
:1011BE00CAE0EDE0EB20F8E8F0EEEAEEE2E5F8E06A
:1011CE00F2E5EBFCEDEEE3EE20EEE1ECE5EDE00A10
:1011DE00003E532C5330362C253032625825303297
:1011EE0062582530326258253032625825303262CC
:1011FE005825303262582C4D414320E0E4F0E5F1A1
:10120E0020F8E8F0EEEAEEE2E5F8E0F2E5EBFCEDD0
:10121E00EEE3EE20EEE1ECE5EDE00A003E454E4455
:10122E000A0044756D705820202020203030203068
:10123E0031203032203033203034203035203036DB
:10124E0020303720303820303920304120304220B5
:10125E0030432030442030452030460A003A2000EA
:10126E000A0044756D70442020202020303020303C
:10127E00312030322030332030342030352030369B
:10128E002030372030382030392030412030422075
:10129E0030432030442030452030460A00457272DB
:1012AE00206B657900526420656570726F6D0A005F
:1012BE005264204D454D0A00526420436F64650A06
:1012CE000044656275674950204F4E0A00446562BE
:1012DE0075674950204F46460A004465627567554A
:1012EE00736572204F6E0A004465627567557365AB
:1012FE0072204F46460A0044656275674D7367203B
:10130E004F6E0A0044656275674D7367204F4646FF
:10131E000A00436F6E666967206C6F636B210A006B
:10132E00577220656570726F6D0A00205361766585
:10133E0020656570726F6D210A00457272204D41F5
:10134E004321004C6F61643E3E002A003C41303127
:10135E003D003C4130323D003C4130333D003C418C
:10136E0030343D003C4130353D003C4130363D008F
:10137E004E4F4950004C494E4B434F4E5452005421
:10138E0052415353004652004E4F4C494E4B00496A
:10139E004E49004E4F4449414700003C21003C530A
:1013AE0030313D003C5330323D003C5330333D0034
:1013BE003C5330343D003C5330353D003C533036C9
:1013CE003D00FF137EFF1383FF138DFF1393FF1357
:0A13DE0096FF139DFF13A1FF13A853
:063805000147000145002F
:10387000C2AFC28E438910758BFF758DB7D2ABD2A4
:043880008ED2AF2213
:03001B00022F10A1
:102F1000C0E0C083C082C0D0C2AFC28E758BFF75C7
:102F20008DB720060675A61E75A6E10545D202E5F9
:102F30004760020547E546D3940140021546054A1D
:102F4000E54A540F7050D20DE54A543F701AD20032
:102F500090668DE0601204F0E0D394B4400A908053
:102F6000007480F0C2AF80FE906688E0600204F0DA
:102F7000906104E0600214F090668EE0D39401400A
:102F800003E014F03005020548E549D39464400499
:102F9000D20680020549E544D3940140021544D28B
:0C2FA0008ED2AFD0D0D082D083D0E032EF
:10088100C291C290D2B5C20A7D027C007F071237A5
:10089100E88F25E525646060097D017F601237A03E
:1008A100D20AE4FDFC7F0B1237E88F25E52530E6FF
:1008B100097D04E4FF1237C4D20A7D017C007F0761
:1008C1001237E88F25E5257008FD7FFF1237A0D28A
:1008D1000A300A03126000C2AFC288C2A8C2AA7558
:1008E10089001232DA906341E0B4FA09A3E064CEE0
:1008F1007003020981E4F52574392525F582E43474
:1009010063F583E4F00525E525B443EC9063417478
:10091100FAF0A374CEF0A374CCF0906347740AF09C
:10092100E4A3F0A304F0A3F090634C7403F0A37468
:10093100CCF090633D74FFF0A3F0A3F0E4A3F0903A
:1009410063587405F0E4F525E5252401FFE433FE41
:1009510074392525F582E43463F583E0FD123857B7
:100961000525E525C3944340DFE4F5A775A61E756B
:10097100A6E1907FF0F0A3F09080007480F080FEFB
:10098100D2AF90634C7403F0A374CCF0E490634B4A
:10099100F01228F1EF6003121EC8C2B51234C7C2AB
:1009A10006123664906358E0C3940350037403F055
:1009B100D20AC20CC20BD293200A077E0E7F9E126E
:1009C10029D7E4906578F0123870C2AFA37408F0AB
:1009D1009062B77424F0E4A3F0906341E09062B9AF
:1009E100F0906342E09062BAF0906343E09062BBA2
:1009F100F0906344E09062BCF0906345E09062BD8A
:100A0100F0906346E09062BEF0754601E490657A2D
:100A1100F0C207C208D2AF75A70775A61E75A6E179
:100A2100200A18AF25FE7D03122AB8E4FF122D1B00
:100A31007E637F78E4FB7D01122B9290668DE060EE
:100A4100037401F0E4906104F0A37455F0A3748180
:100A5100F0E4F548E4F549906104E0700312377061
:100A610090668EE0B401119080007410F0E49066FD
:100A71008EF0D20AD20BD20C908008E0F52530E43A
:100A810005D2077410F0E52530E508D209908008F9
:100A91007420F0E52530E608D2089080087440F013
:100AA100E548D394034023908002E4F0908001F064
:100AB100908000F0E548D39406400FE4F548C20366
:100AC10090657AF07546011236649080A0E070035B
:100AD1001233D39080B8E0700312344D9080D0E08F
:100AE10070031235A4908000E070133007101226B5
:100AF100EC906334EFF0D394004003120026908011
:100B010002E07006908000E06005D205020A55C23D
:100B110005E4F548906104E06003020A55300912CA
:100B2100122586906334EFF0D394004005E0FF1264
:100B31000022200803020CB4122411906334EFF058
:100B41007003020A55906378E054BF247F7003025A
:100B51000C17147003020BEF24026003020C4A20ED
:100B61000A077E0E7FA71229D7300E7920037690CF
:100B71006350E07006906354E0605B906684E0FF30
:100B8100906350E0B50724906685E0FE906351E0E4
:100B9100B50618906686E0FE906352E0B5060C90AB
:100BA1006687E0FE906353E06E602B906354E06FC4
:100BB1007033906685E0FF906355E0B50727906636
:100BC10086E0FF906356E0B5071B906687E0FF90D3
:100BD1006357E0B5070F90657A7401F012001E7536
:100BE1004601020CB490668474FFF0020CB4906666
:100BF1008DE060037401F090667CE0FF90637AE021
:100C01006F6003020CB490667CE004F0E4F546905A
:100C11006578F0020CB4300303020CB4906347E032
:100C21007003020A55123899D203E4F546906578AB
:100C3100F090668804F0E490667BF0A3F0200A73DC
:100C41007E0E7FB51229D7806A90668DE0600374AD
:100C510001F0300352906378E020E74B90637AE033
:100C6100FF90667BE0FE6F600D906683E07007EE9B
:100C7100146F703F801390667BE004F0906334E062
:100C8100FFD3940440031235409060007482F0A3B6
:100C91007401F090637AE0906002F07E607F007DE5
:100CA10003123358020A55300E0920030690668458
:100CB10074FFF0200303020D69E546706B122FAC3F
:100CC100EF60207E647F78906479E02404FD123324
:100CD10058906683E06003020A55906358E0F54638
:100CE100020A55906688E0D3943C403C906683E0CC
:100CF100703690668804F09062B6E0702B122C6614
:100D0100E4906478F0A37412F090667CE090647AC9
:100D1100F0A374FDF090610763A20190647C63A26B
:100D2100017F12122196809B123884EF601590602A
:100D3100007483F0E4A3F07E607F007D02123358DB
:100D4100020A55E54664016003020A55906578E0A0
:100D510004F0E0C394055003020CC4C203E490659F
:100D61007AF012001E020A55E54664016003020A88
:100D71005590657AE014604024FE603C14700302D3
:100D81000E5124046003020A55E4F548200E139025
:100D9100657A7404F0906578E05401F075460102BB
:100DA1000A55E490657AF090657804F07546C8902C
:100DB100668474FFF0020A55906684E07003020EA7
:100DC100409064787480F090647A7401F0E4A3F048
:100DD100A304F0A37430F0A3747BF0E4F525747FD1
:100DE1002525F582E43464F583747DF0748025252E
:100DF100F582E43464F583E4F0E525240790647911
:100E0100F07C667D8490634CE0FAA3E0FB7F0212E4
:100E110031567E647F78E5252409FD1233589066AA
:100E210083E0601B123899D203E4F546906578F0AF
:100E310090668804F0E490667BF0A3F0020A559076
:100E4100657A7404F0906358E02432F546020A553D
:100E51009080027410F0754603906578E06401FF9C
:100E6100F090657A7401F0EF7019906354E06013AB
:100E7100FCA3E0FDA3E0FEA3E0FF906684121B3219
:100E8100020A55906350E0FCA3E0FDA3E0FEA3E05D
:0C0E9100FF906684121B32020A5580FE9E
:010E9D002232
:10002600906379E0B444047F0180027F0090637896
:10003600E0B447047E0180027E00EE5F604A906372
:1000460041E090637AF0906342E090637BF09063C6
:1000560043E090637CF0906344E090637DF09063AE
:1000660045E090637EF0906346E090637FF0906396
:10007600797452F09062B063A2019080A863A201E5
:100086007F06122196020877906334E0C3940850E5
:1000960003020880906341E0FF90637AE06F60039B
:1000A600020880906342E0FF90637BE06F6003028A
:1000B6000880906343E0FF90637CE06F6003020872
:1000C60080906344E0FF90637DE06F6003020880E8
:1000D600906345E0FF90637EE06F600302088090C6
:1000E6006346E0FF90637FE06F60030208809063E1
:1000F60079E0B444159062B0E0B4FF0E63A20190BB
:1001060080A863A2017F0612219690668DE06003A7
:100116007401F090668E7464F09063797452F09076
:100126006378E0646D60030202A37BFF7A0E79BFF9
:1001360012144A7BFF7A0E79D9906341E0F52EA31B
:10014600E0F52FA3E0F530A3E0F531A3E0F532A307
:10015600E0F53312144A752EFF752F0F753036757C
:1001660031FF75320F7533427BFF7A0F790F121408
:100176004A7BFF7A0F794B12144A7BFF7A0F79B1CB
:1001860012144A7BFF7A0F79DE906347E0F52EA3BF
:10019600E0F52FA3E0F530A3E0F53112144A7BFF1A
:1001A6007A107908906350E0F52EA3E0F52FA3E0CE
:1001B600F530A3E0F53112144A7BFF7A10793690B8
:1001C6006354E0F52EA3E0F52FA3E0F530A3E0F5A8
:1001D6003112144A7BFF7A10796490633DE0F52E64
:1001E600A3E0F52FA3E0F530A3E0F53112144A7B26
:1001F600FF7A107987906339E0F52EA3E0F52FA3F7
:10020600E0F530A3E0F53112144A7BFF7A1079A4A9
:10021600906358E0F52E12144A7BFF7A1079CE12BD
:10022600144A7BFF7A1079F7A20EE433F52E1214E6
:100236004A7BFF7A117927906683E0F52E12144ADD
:100246007BFF7A11795290668DE0F52E12144A7B67
:10025600FF7A1179859062B6E0F52E12144A7BFF7B
:100266007A1179B3A201E433F52E12144A7BFF7A90
:100276001179DF90667DE0F52EA3E0F52FA3E0F57A
:1002860030A3E0F531A3E0F532A3E0F53312144ACA
:10029600122DC57BFF7A12792A12144A22906378AE
:1002A600E0644C70527E127F301229D7906380E052
:1002B600F526A3E0F527E4F5287D03AF27AE261241
:1002C6002AB87E127F6B1229D7AE26AF27E4FB7DB4
:1002D60010122B927E127F6E1229D774102527F5E5
:1002E60027E43526F5260528E528C3941040CA7E5E
:1002F600127F6E1229D722906378E0646C705CF5E9
:100306002A7E127F701229D7E4F529AF2A7E007D56
:1003160003122AB87E127F6B1229D7E4F528A82A81
:10032600E6FF74822528F582E43463F583EFF00551
:100336002A0528E528B410E67E637F82E4FB7D105B
:10034600122B927E127F6E1229D70529E529C394B6
:100356000840B87E127F6E1229D722906378E06437
:100366004B7061F528746A2528F582E43463F583B9
:10037600E06032746A2528F582E43463F583E0F49C
:100386006023746A2528F582E43463F583E0FF74FC
:10039600802528F582E43463F583E0B50710052847
:1003A600E528B408C09061047432F00208779063BF
:1003B600787421F0300A030208777E127FAB122987
:1003C600D7020877906378E0B4521A200A077E12A3
:1003D6007FB31229D79063787472F07E637F787D3D
:1003E600081231DA22906378E064497045200A07E2
:1003F6007E127FBE1229D7906380E0F526A3E0F532
:1004060027E4F528852782852683E0FF7482252840
:10041600F582E43463F583EFF00527E527700205DE
:10042600260528E528B480DC7E637F787D8A123134
:10043600DA22906378E064437079A3E064527046F0
:10044600200A077E127FC61229D7906380E0F52620
:10045600A3E0F527E4F528852782852683E493FF24
:1004660074822528F582E43463F583EFF00527E5E9
:1004760027700205260528E528B480DB7E637F7891
:100486007D8A1231DA22906379E0645760030208AC
:1004960080906380E0F526A3E0F52774822528F591
:1004A60082E43463AD82FC7B80AF27AE2612373CF4
:1004B600020877906378E06444600302054A90631B
:1004C60080E0FF64447003020877EFB4310CC20A7F
:1004D6007E127FCF1229D7020877906380E0B4306E
:1004E6000CD20A7E127FDB1229D70208779063802E
:1004F600E0B4320CD20B7E127FE81229D7020877BD
:10050600906380E0B4330CC20B7E127FF61229D7BB
:10051600020877906380E0B4340CD20C7E137F051A
:100526001229D7020877906380E0B4350CC20C7E9E
:10053600137F121229D7020877906380E0FF12001A
:1005460021020877906104E07013200A077E137F6A
:10055600201229D79063787421F0020877906104FD
:100566007432F0906378E0FFB4510A908000748092
:10057600F0C2AF80FEEF64577045200A077E137FF6
:100586002E1229D7906381E0906334F0E4F5289029
:100596006334E0FFE528C39F400302087774822591
:1005A60028F582E43463F583E0FF906380E0252834
:1005B60024AFF582E43461F583EFF0052880D0900E
:1005C6006378E064536003020679200A077E137F8E
:1005D600391229D7906341E0FF9061B8E06F703C13
:1005E600906342E0FF9061B9E06F7030906343E042
:1005F600FF9061BAE0B50724906344E0FF9061BBC9
:10060600E0B50718906345E0FF9061BCE0B5070CC4
:10061600906346E0FF9061BDE06F6016906378746A
:1006260021F0300A030208777E137F481229D70289
:100636000877E4F528E4F549AF28FE74AF2528F5D8
:1006460082E43461F583E0FD1238570528E528C3B6
:1006560094FE40E19080007480F0C2AFE4907FF099
:10066600F0A3F0907FFD74AAF0A374FFF0A3745575
:10067600F080FE906378E0644F704C906380E0F504
:1006860026A3E0F527E5274526700A200A077E13EC
:100696007F511229D7200A077E137F581229D7E4E3
:1006A600F52874822528F582E43463F583E08527EE
:1006B60082852683F00527E527700205260528E5AD
:1006C60028B480DE020877906378E0FFB44527906F
:1006D60080007480F0906380E0FDA3E0907FF0CD11
:1006E600F0A3EDF0C2AF907FFD74AAF0A374FFF003
:1006F600A37455F080FEEF6465600302087790638B
:1007060080E0FFA3E0907FF0CFF0A3EFF0E4F526C2
:10071600F527D3907FF1E09527907FF0E09526406E
:1007260020E4F5492527FFE5263401FE8527828545
:100736002683E0FD1238570527E527700205268037
:10074600D17E137F5A1230D1EF4E602012000390F3
:100756006347EFF0120003906348EFF01200039036
:100766006349EFF012000390634AEFF07E137F6057
:100776001230D1EF4E6020120003906350EFF0125A
:100786000003906351EFF0120003906352EFF012F2
:100796000003906353EFF07E137F661230D1EF4E65
:1007A6006020120003906354EFF01200039063552B
:1007B600EFF0120003906356EFF0120003906357B8
:1007C600EFF07E137F6C1230D1EF4E6020120003E3
:1007D60090633DEFF012000390633EEFF0120003CA
:1007E60090633FEFF0120003906340EFF07E137FBB
:1007F600721230D1EF4E6020120003906339EFF091
:1008060012000390633AEFF012000390633BEFF09F
:1008160012000390633CEFF07E137F781230D1EF25
:100826004E6008123607906358EFF0E4F528E4F5B9
:1008360049E5282401FFE433FE74392528F582E4CE
:100846003463F583E0FD1238570528E528C3944341
:1008560040DC9080007480F0C2AFE4907FF0F0A39B
:10086600F0907FFD74AAF0A374FFF0A37455F08096
:0A087600FE7E637F787D081231DA00
:010880002255
:10370400AE07EEC39430400BEED394395005EE244B
:10371400D0FF22EEC39461400BEED394665005EEC5
:1037240024A9FF22EEC39441400BEED394465005E6
:08373400EE24C9FF22AF0622BA
:10383D009062AFE004F070069062AEE004F090622A
:0A384D00AEE0FEA3E0FF12382122D6
:1000030012383D123704EFC454F0FEC00612383DD7
:08001300123704D0E02FFF2298
:10360700E49068AFF012383D9068B0EFF0C39430A3
:103617004018E0FFD3943950119068AFE02407F5C4
:1036270082E43461F583EFF080119068AFE02407FE
:10363700F582E43461F583E4F0800C9068AFE00430
:10364700F0E0D3940840BE752E00752F007530004A
:0C365700E4F5317B017A61790712226DE5
:013663002244
:0430D1008E2B8F2C87
:1030D5009062AEE4F0A374FFF012383DEF606EF439
:1030E500606B852C82852B83E493B507EC752D01E8
:1030F500E52C252DF582E4352BF583E493602590A9
:1031050062AFE0252DFF9062AEE03400FE1238215B
:10311500E52C252DF582E4352BF583E493B50704DD
:10312500052D80CCE52C252DF582E4352BF583E4A2
:103135009370A6E52D24FFFFE434FFFE9062AFE017
:103145002FF09062AEE03EF07E007F0122E4FEFFAC
:013155002257
:1028F1007E137FA91230D1EF4E70037F01227E1328
:102901007FAC1230D1EF4E600C12383DEF24D02451
:10291100FF920E8002D20E7E137FB21230D1EF4EA3
:10292100600C12383DEF24D0906683F08005E4906E
:102931006683F07E137FB81230D1EF4E600C1238EF
:102941003DEF24D090668DF08005E490668DF07E99
:10295100137FBE1230D1EF4E600C12383DEF24D000
:102961009062B6F08005E49062B6F07E137FC412E7
:1029710030D1EF4E600C12383DEF24D024FF92018C
:102981008002C20190634163A20190667D63A2014E
:102991007F0612219630013B7E137FCA1230D1EFA0
:1029A1004E603012000390667DEFF01200039066D6
:1029B1007EEFF012000390667FEFF0120003906645
:1029C10080EFF0120003906681EFF0120003906631
:0629D10082EFF07F0022FE
:101EC800C201E490668DF0D20EC204906683F09051
:101ED80062B6F090634163A20190667D63A2017FC0
:101EE80006122196E4F526E52675F003A424D0F51C
:101EF80082E43413F583E493FB740193FA74029338
:101F0800F91219FF70030220BAE4F527F528FD74C9
:101F18002F2DF582E43461F583E0FF70030220B5CC
:101F2800E52675F003A424D0F582E43413F583E4A0
:101F380093FB740193FA740293F9852782758300E1
:101F4800121A18FEEFB5060875280105270220B1F8
:101F5800E52870030220B1EE60030220ACE52624D8
:101F6800FE60281470030220941470030220981451
:101F780070030220A01470030220A4240560030249
:101F880020B590668D7401F00220B5D201742F2D12
:101F9800F582E43461F583E0FF642D70030220B517
:101FA800123704EFC454F0FC74302DF582E4346128
:101FB800F583E0FF123704EF2C90667DF074312D25
:101FC800F582E43461F583E0FF123704EFC454F07E
:101FD800FC74322DF582E43461F583E0FF12370496
:101FE800EF2C90667EF074332DF582E43461F5832E
:101FF800E0FF123704EFC454F0FC74342DF582E48A
:102008003461F583E0FF123704EF2C90667FF0749B
:10201800352DF582E43461F583E0FF123704EFC40F
:1020280054F0FC74362DF582E43461F583E0FF1238
:102038003704EF2C906680F074372DF582E4346114
:10204800F583E0FF123704EFC454F0FC74382DF523
:1020580082E43461F583E0FF123704EF2C90668147
:10206800F074392DF582E43461F583E0FF1237040A
:10207800EFC454F0FC743A2DF582E43461F583E042
:10208800FF123704EF2C906682F08021D204801D65
:102098009066837401F08015C20E80119062B67448
:1020A80001F08009E4F528F5270D021F170526021F
:0220B8001EEF19
:0120BA002203
:1036BD00906579E0C3947C503D906579E0FE04F00F
:1036CD0074B72EF582E43462F583EFF0BF0A2790CC
:1036DD006579E0FF04F074B72FF582E43462F58369
:1036ED00E4F0906579E0FF12325C9065797408F032
:0736FD009062B8E004F02226
:103664009080007480F090633963A201F583F58241
:1036740063A2017F0812219690634163A2019080A6
:103684008863A2017F0A122196908092E4F0A374C9
:1036940032F0A37401F090634BE0FF9080B1F0909E
:1036A40080E1EFF09080957455F0A3F09080007461
:0936B40001F09080097470F0220D
:1033D300908009E04410F09080A0E0706C9080A190
:1033E3007482F09080A874FFF0A3F0A3F0A3F07FA1
:1033F300039080AEEFF07FCBA3EFF07F039080AC20
:10340300EFF0A374CBF09080007402F09068A312E5
:103413001B3E000000009068A3E0908040F090689D
:10342300A4E0908041F09068A5E0908042F090681D
:10343300A6E0908043F0A3E4F0A3F0A3F0A3F09000
:093443008018F0A3F0A3F0A3F03F
:01344C00225D
:1035A400908009E04440F09080D17482F090634CA4
:1035B400E0FF9080DEF090634DE0FF9080DFF090BC
:1035C40080027402F09068A7121B3E000000009075
:1035D40068A7E0908058F09068A8E0908059F09037
:1035E40068A9E090805AF09068AAE090805BF0A30C
:1035F400E4F0A3F0A3F0A3F0908030F0A3F0A3F0E4
:02360400A3F031
:0136060022A1
:10344D00908009E04420F09080B8E0706C9080B9D5
:10345D007482F07F039080C6EFF07FCDA3EFF07FF5
:10346D00039080C4EFF0A374CDF09080C074FFF092
:10347D00A3F0A3F0A3F09080017402F09068AB125A
:10348D001B3E000000009068A7E090804CF0906813
:10349D00A8E090804DF09068A9E090804EF0906883
:1034AD00AAE090804FF0A3E4F0A3F0A3F0A3F09076
:0934BD008024F0A3F0A3F0A3F0B9
:0134C60022E3
:103156008C268D27A907EAFDE975F018A424ACFF93
:10316600E5F034808F82F583EDF0EBFDE975F0181C
:10317600A4FFAEF024ACFBEE34808B82F583A3ED86
:10318600F08527828C83E0FDEF24A8FFEE3480FED5
:103196008F82F583EDF08527828C83A3E08F828E64
:1031A60083A3F0852782852683A3A3E0FDE975F036
:1031B60018A424A8FFE5F03480FE8F82F583A3A32C
:1031C600EDF08527828C83A3A3A3E08F828E83A351
:0431D600A3A3F0229D
:0631DA008D2BAB07AA06D5
:1031E0009068A3E0FCA3E0FDA3E0FEA3E0F52F8E32
:1031F0002E8D2D8C2CAE02AF038E838F8263A201A5
:10320000E52E540744C0F583852F8263A201AF2BBE
:103210001221FF908000E020E5F9E4FCFDFEE52F9F
:10322000252BF52FEE352EF52EED352DF52DEC3524
:103230002CF52C908040E52CF0A3E52DF0A3E52E95
:10324000F0A3E52FF09080007420F0AF2FAE2EADEC
:0B3250002DAC2C9068A3121B32AF2B9A
:01325B002250
:063358008D26AB07AA065A
:10335E009068A7E0FCA3E0FDA3E0FEA3E0F52A8EB3
:10336E00298D288C27AE02AF038E838F8263A20134
:10337E00E529540744D0F583852A8263A201AF263E
:10338E001221FFE4FCFDFEE52A2526F52AEE35295D
:10339E00F529ED3528F528EC3527F527908058E5E9
:1033AE0027F0A3E528F0A3E529F0A3E52AF0908005
:1033BE00027420F0AF2AAE29AD28AC279068A71270
:0433CE001B32AF26D9
:0133D20022D8
:022D1B008F2601
:102D1D00908001E030E5037F00229068ABE0FCA3DA
:102D2D00E0FDA3E0FEA3E0F52A8E298D288C2790E7
:102D3D00667D63A201E529540744C8F583852A827F
:102D4D0063A2017F06122215E52A2406F52AE43531
:102D5D0029F529E43528F528E43527F52790657BF5
:102D6D0063A201E529540744C8F583852A8263A22D
:102D7D0001AF26122215E4FCFDFEE52A2526F52AD3
:102D8D00EE3529F529ED3528F528EC3527F5279071
:102D9D00804CE527F0A3E528F0A3E529F0A3E52A6B
:102DAD00F09080017420F0AF2AAE29AD28AC2790A9
:072DBD0068AB121B32AF26C8
:012DC40022EC
:1026EC009081E0E0F526052605260526052605261B
:1026FC0005260526052605260526908010E0F529D9
:10270C00A3E0F52AA3E0F52BA3E0F52C9081E1E002
:10271C00F526052605260526052605260526052665
:10272C00052605260526908014E0F52DA3E0F52E50
:10273C00A3E0F52FA3E0F530E52FB52B08E530B578
:10274C002C037F0022E4F526E52F540744E0F583A3
:10275C0085308263A20190637863A2017F08122204
:10276C002D90637A63A2019062B063A2017F06127E
:10277C002196906378E0F527A3E0F528E4F5269000
:10278C006378E0702AA3E024F8F526E52F5407447B
:10279C00E0F58385308274082582F582E43583F573
:1027AC008363A20190637863A201AF2612222DAE3F
:1027BC0027E4FCFDE5302528F530E52F3EF52FED1F
:1027CC00352EF52EEC352DF52D908014E52DF0A33E
:1027DC00E52EF0A3E52FF0A3E530F09080007440D7
:0327EC00F0AF2625
:0127EF0022C7
:102411009081E6E0F52605260526052605260526F2
:1024210005260526052605260526908028E0F5299E
:10243100A3E0F52AA3E0F52BA3E0F52C9081E7E0DA
:10244100F526052605260526052605260526052643
:1024510005260526052690802CE0F52DA3E0F52E16
:10246100A3E0F52FA3E0F530E4F526E52FB52B0A1F
:10247100E530B52C05C20802256BE52F540744F061
:10248100F58385308263A20190637863A2017F089E
:1024910012222D906378E0F527A3E0F528E5284581
:1024A1002770099080027410F07F0022906684E00A
:1024B100FFF4602D90637AE06F7076906685E0FF9F
:1024C10090637BE06F706A906686E0FF90637CE0CA
:1024D1006F705E906687E0FF90637DE06F602280A1
:1024E1005090637AE0906684F090637BE09066851B
:1024F100F090637CE0906686F090637DE090668763
:10250100F0906378E0702AA3E024F8F526E52F54D3
:102511000744F0F58385308274082582F582E4351D
:1025210083F58363A20190637863A201AF2612222F
:102531002DAE27E4FCFDE5302528F530E52F3EF5ED
:102541002FED352EF52EEC352DF52DAF2CAE2BAD17
:102551002AAC29AB30AA2FA92EA82DD3121B2140BA
:10256100099080027410F07F002290802CE52DF0FC
:10257100A3E52EF0A3E52FF0A3E530F090800274DF
:0425810040F0AF2651
:012585002233
:102586009081E3E0F526052605260526052605267F
:102596000526052605260526052690801CE0F52934
:1025A600A3E0F52AA3E0F52BA3E0F52C9081E4E067
:1025B600F5260526052605260526052605260526CD
:1025C600052605260526908020E0F52DA3E0F52EAC
:1025D600A3E0F52FA3E0F530E4F526E52FB52B0AA9
:1025E600E530B52C05C2090226D1E52F540744E88B
:1025F600F58385308263A20190600463A2017F0E99
:10260600122243906004E0F527A3E0F52890600CC1
:10261600E0FFF4604590667DE0FEEF6E706EA3E02D
:10262600FF90600DE06F706490667FE0FF90600E33
:10263600E06F7058906680E0FF90600FE06F704C1E
:10264600906681E0FF906010E06F7040906682E0D7
:10265600FF906011E06F60048032D2D9906004E090
:10266600702AA3E024F2F526E52F540744E8F58303
:10267600853082740E2582F582E43583F58363A264
:102686000190600463A201AF26122243AE27E4FC48
:10269600FDE5302528F530E52F3EF52FED352EF5F5
:1026A6002EEC352DF52DAF2CAE2BAD2AAC29AB304B
:1026B600AA2FA92EA82DD3121B215006E52845279F
:1026C60070099080017410F07F0022908020E52D23
:1026D600F0A3E52EF0A3E52FF0A3E530F0908001FE
:0526E6007440F0AF2676
:0126EB0022CC
:0429D7008E2B8F2C88
:1029DB009068A3E0FCA3E0FDA3E0FEA3E0F5328E3C
:1029EB00318D308C2FE532FFE5315407FEE42FF5A6
:1029FB002EEE34C0F52D852E82F5837423F0052E33
:102A0B00E52E7002052D532DC7F582852D83740A93
:102A1B00F0052EE52E7002052D532DC790634163F3
:102A2B00A201852D83852E8263A2017F061221FFD1
:102A3B007406252EF52EE4352DF52D852B83852C4F
:102A4B008263A201852D83852E8263A2011221E36D
:102A5B00908000E020E5F9E4FCFDFE9068A3E0F82F
:102A6B00A3E0F9A3E0FAA3E02FFFEE3AFEED39FD68
:102A7B00EC38FCEF2408FFE43EFEE43DFDE43CFCB7
:102A8B009068A3121B329068A3E0908040F090688E
:102A9B00A4E0908041F09068A5E0908042F09068AF
:0C2AAB00A6E0908043F09080007420F0C2
:012AB70022FC
:062B92008E2B8F2C8D2D0F
:102B98009068A3E0FCA3E0FDA3E0FEA3E0F5338E7C
:102BA800328D318C30E533FFE5325407FEE42FF5E2
:102BB8002FEE34C0F52E852F82F5837423F0052F70
:102BC800E52F7002052E532EC7F582852E83EBF074
:102BD800052FE52F7002052E532EC790634163A27F
:102BE80001852E83852F8263A2017F061221FF743F
:102BF80006252FF52FE4352EF52E852B83852C827F
:102C080063A201852E83852F8263A201AF2D122135
:102C1800FF908000E020E5F97408252DF52DFFE4EC
:102C2800FCFDFEE5332FF533EE3532F532ED353167
:102C3800F531EC3530F530908040E530F0A3E531E2
:102C4800F0A3E532F0A3E533F09080007420F0AFF4
:0D2C580033AE32AD31AC309068A3121B32A8
:012C6500224C
:02325C008F3FA2
:10325E009068A3E0FCA3E0FDA3E0FEA3E0F5438E9F
:10326E00428D418C40E543FFE5425407FEE42FFFBB
:10327E00EE34C09062B763A201F5838F8263A20120
:10328E00AF3F1221FF908000E020E5F9E4FCFDFE47
:10329E00E543253FF543EE3542F542ED3541F54127
:1032AE00EC3540F540908040E540F0A3E541F0A3B9
:1032BE00E542F0A3E543F09080007420F0AF43AEFA
:0B32CE0042AD41AC409068A3121B32DF
:0132D90022D2
:062AB8008E2B8F2CAB05F4
:102ABE009068A3E0FCA3E0FDA3E0FEA3E0F5328E58
:102ACE00318D308C2FE532FFE5315407FEE42FF5C2
:102ADE002EEE34C0F52D852E82F5837423F0052E4F
:102AEE00E52E7002052D532DC7F582852D83EBF053
:102AFE00052EE52E7002052D90634163A201852DF2
:102B0E0083852E8263A2017F061221FF7406252E75
:102B1E00F52EE4352DF52D532DC7E52B852E82850B
:102B2E002D83F0052EE52E7002052D532DC7F5824F
:102B3E00852D83E52CF0052EE52E7002052D532DE7
:102B4E00C7908000E020E5F9E532240AF532E4353D
:102B5E0031F531E43530F530E4352FF52F908040E6
:102B6E00E52FF0A3E530F0A3E531F0A3E532F090C8
:102B7E0080007420F0AF32AE31AD30AC2F9068A330
:032B8E00121B32E5
:012B91002221
:10382100E5D220E0FBC2AF438E2075D2028F828E9B
:0B38310083E0FFE4F5D2538EDFD2AF3E
:01383C002269
:10385700E5D220E0FBC2AF43D2028F828E83EDF028
:0938670075D25063D250D2AF2299
:1032DA00E4FDED2401FFE433FE12382174392DF5A3
:1032EA0082E43463F583EFF00DBD3FE6E4FDED249F
:1032FA007FFFE433FE123821742F2DF582E4346106
:10330A00F583EFF0742F2DF582E43461F583E070D4
:10331A001B742F2DF582E43461F5837420F0743028
:10332A002DF582E43461F583E4F080040DBD80BE9E
:10333A00E49061AEF0FDEDFF7E0012382174AF2DEE
:0D334A00F582E43461F583EFF00DBDFEE97E
:013357002253
:02373C008B2BD5
:10373E00A2AF921BC2AF85A22C53A2FE8E838F82A4
:10374E0005A28C838D82740912225BE52B53A2FE97
:10375E0043A22012225D53A2DF852CA2A21B92AFA0
:01376E00FF5B
:01376F002237
:1037E800A2AF921BC2AF8C838D82EF12225B43A2E1
:0C37F8002012225D53A2DFA21B92AFFF43
:0138040022A1
:0237A0008F2672
:1037A200A2AF921BC2AFE4F5838D82740612225B34
:1037B200E52643A22012225D53A2DFA21B92AF7F15
:0137C2000105
:0137C30022E3
:0237C4008F264E
:1037C600A2AF921BC2AFE4F5838D82740A12225B0C
:1037D600E52643A22012225D53A2DFA21B92AF7FF1
:0137E60001E1
:0137E70022BF
:1020BB00A907E7FFA805EF93C3966008403B74FCA4
:1020CB002FFF80F00F08EF93C3966008402B74FB33
:1020DB002FFF80E00F08EF93C3966008401B74FA44
:1020EB002FFF80D00F08EF93D3966008400B74F945
:1020FB002FFF80C01F1F1F1F1FEF54FEF80303F796
:10210B00E893FC08E893FD08E893FE08E893FF22A8
:10211B0009E993C39D6008402974FB29F980F109F3
:10212B00E993C39E6008401A74FA29F980E209E921
:10213B0093D39F6008400B74F929F980D3191919AF
:10214B001919E9C313C313FF22740093F8ECC39856
:10215B004024701F740193F8EDC3984019701474E8
:0E216B000293F8EEC398400E7009740393F8C7
:10217900EFC39840037F00227F0122EDF8E6F008C3
:10218900A3DFFA22EDF8E0F608A3DFFA22E0A36361
:10219900A201F0A363A201DFF475A20022E0A36308
:1021A900A201F0A363A201E0A363A201F0A363A2C9
:1021B90001E463A201F0A363A201DFE175A2002299
:1021C900E0A363A2016DFE936CFDEE058393FC15FC
:1021D9008363A201DFEA75A200227F00E493A3636F
:1021E900A201F00F600CA3E583C2E3F58363A201AA
:1021F90080EA75A20022E0A363A201F0A3E583C2ED
:10220900E3F58363A201DFEE75A20022E0A363A2D6
:1022190001F0A3E583C2E4D2E3F58363A201DFEC15
:1022290075A20022E583C2E3F583E0A363A201F06E
:10223900A363A201DFEE75A20022E583C2E4D2E323
:10224900F583E0A363A201F0A363A201DFEC75A209
:102259000022F922C002C004C00612FFF0D006D045
:0422690004D0022279
:101744005452414E5A0053545245414D0052545341
:101754000044454C4159004D4F4445004C494D49C6
:10176400540053495A45004C454E47544800455689
:10177400454E504152495459004F444450415249F6
:101784005459004B56545F494E004B56545F4F55C5
:101794005400574149540053544F5000003E2A2CE2
:1017A400312CCFE0F0E0ECE5F2F0FB20E0F1E8EDE5
:1017B400F5F0EEEDEDEEE3EE20EFEEF0F2E00A00F0
:1017C4003E4C2C4930312C256C752CD1EAEEF0EED0
:1017D400F1F2FC20EEE1ECE5EDE02C35302C31307B
:1017E400302C3330302C3630302C313230302C32F7
:1017F4003430302C343830302C393630302C3139C8
:101804003230302C33383430302C35373630302CBD
:101814003131353230300A003E422C4930322C25E9
:1018240062752CC2FBF1F2E0E2EBFFF2FC205254B1
:101834005320EFF0E820EFE5F0E5E4E0F7E50A00F7
:101844003E532C4930332C2562752CC7E0E4E5F077
:10185400E6EAE020F1F2E0F0F2E020EFE5F0E5E482
:10186400E0F7E8282A3130ECF1290A003E422C49FD
:1018740030342C2562752CD0E5E6E8EC20EFE5F059
:10188400E5E4E0F7E8203720E1E8F20A003E422CE4
:101894004930352C2562752CCFE5F0E5E4E0F7E01E
:1018A40020F120EAEEEDF2F0EEEBFCEDFBEC20E1B2
:1018B400E8F2EEEC0A003E422C4930362C256275E3
:1018C4002CCAEEEDF2F0EEEBFCEDFBE920E1E8F2E0
:1018D400202D20F7E5F2EDEEF1F2FC0A003E532C48
:1018E4004930372C2562752CC4EEF1F2E0E2EAE0CF
:1018F40020EFF0E820EFF0E8E5ECE5204E20E1E011
:10190400E9F220283C313236290A003E532C493072
:10191400382C2562752CC4EEF1F2E0E2EAE020EF07
:10192400F0E820EFE0F3E7E520EFF0E8E5ECE02075
:10193400282A3130ECF1290A003E532C4930392C45
:101944002562752CC4EEF1F2E0E2EAE020EFF0E863
:1019540020EFF0E8E5ECE520E1E0E9F2E0202830D2
:101964002DEDE5F220EAEEEDF2F0EEEBFF290A00B0
:101974003C21003C4930313D003C4930323D003C83
:101984004930333D003C4930343D003C4930353D1D
:10199400003C4930363D003C4930373D003C49303D
:1019A400383D003C4930393D000AC1F3F4E5F020EC
:1019B400E7E0EDFFF221000A4F55543E000A46725B
:1019C400616D65206572726F722120003C00FF1703
:1019D40044FF174AFF1751FF1755FF175BFF1760A6
:1019E400FF1766FF176BFF1772FF177DFF1787FF3F
:0B19F400178EFF1796FF179BFF17A030
:10380B0052668F0000000000000000000000000066
:05381B000000000000A8
:0100210022BC
:03002300022E6E3C
:0B2E6E00C0E0C083C082C0D075D01847
:102E7900309821754701AF99D29174A1250EF58239
:102E8900E43466F583EFF0050EE50C6005B51F0225
:102E9900D219C298309965301260301807309704FA
:102EA900D20F8056E510C3950D400AC212C290D2C6
:102EB9001AD2968045AF10051074A12FF582E4341B
:102EC90067F583E0F51330151953137F3010282067
:102ED900D008201322631380801D30131A631380D6
:102EE9008015301012E5135213301306A2D0929BAD
:0E2EF9008005A2D0B3929B851399C299D2AFE7
:092F0700D0D0D082D083D0E0329A
:101C70009068A174FFF0A374B8F0C218E4F509C22B
:101C800015C210C213750840750F05F50C9068AFAA
:101C9000F09068AFE075F003A424D2F582E4341923
:101CA000F583E493FB740193FA740293F91219FF1C
:101CB0007003021EC7E49068B1F0A3F09068B0F022
:101CC0009068B0E0242FF582E43461F583E0FF7082
:101CD00003021EBE9068AFE075F003A424D2F58223
:101CE000E43419F583E493FB740193FA740293F9D5
:101CF0009068B1E0F582758300121A18FEEFB50600
:101D00000F9068B27401F09068B1E004F0021EB563
:101D10009068B2E07003021EB5EE6003021EAC9044
:101D200068AFE0B40E004003021EBE901D32F828DA
:101D30002873021D5C021DA9021DAE021DB3021D07
:101D4000E2021E18021E18021E18021E46021E4C37
:101D5000021EBE021EBE021E50021E7E9068B0E031
:101D6000242FF9E43461FA7B01C0031B8B2E752FFD
:101D700000753000E4F531D00312226D9068B31283
:101D80001B329068B3E0F8A3E0F9A3E0FAA3E0FB0C
:101D90007F007E8C7D0A7C00121A81121B139068D2
:101DA000A1EEF0A3EFF0021EBEC216021EBED218B4
:101DB000021EBE9068B0E0242FF9E43461FA7B0182
:101DC000C0031B8B2E752F00753000E4F531D00356
:101DD00012226D9068B3121B329068B6E0F50902CA
:101DE0001EBE9068B0E0FF242FF582E43461F583D5
:101DF000E0B43702D21574302FF582E43461F583F4
:101E0000E0FFB44E04C2108002D210EF64456003BC
:101E1000021EBED213021EBE9068B0E0242FF9E469
:101E20003461FA7B01C0031B8B2E752F00753000C7
:101E3000E4F531D00312226D9068B3121B32906822
:101E4000B6E0F5088078D210D2138072D210806E7E
:101E50009068B0E0242FF9E43461FA7B01C0031BE1
:101E60008B2E752F00753000E4F531D00312226DF2
:101E70009068B3121B329068B6E0F50F804090680E
:101E8000B0E0242FF9E43461FA7B01C0031B8B2EF0
:101E9000752F00753000E4F531D00312226D906883
:101EA000B3121B329068B6E0F50C8012E49068B271
:101EB000F09068B1F09068B0E004F0021CC0906847
:071EC000AFE004F0021C91E9
:011EC70022F8
:102DC5007BFF7A1779A112144A9068A1E0FEA3E06F
:102DD500FFC3E49FFFE49EFEAB07FA3395E0F9F8E5
:102DE5007F007E8C7D0A7C00121A818F318E308D9A
:102DF5002F8C2E7BFF7A1779C412144A7BFF7A1821
:102E0500791CA218E433F52E12144A7BFF7A18793F
:102E15004485092E12144A7BFF7A187970A215E4AD
:102E250033F52E12144A7BFF7A187991A210E433F8
:102E3500F52E12144A7BFF7A1879BAA213E433F5FA
:102E45002E12144A7BFF7A1879E185082E12144A4E
:102E55007BFF7A19790F850F2E12144A7BFF7A1999
:092E6500793D850C2E12144A225D
:1027F0007E197F741230D1EF4E70037F01227E1953
:102800007F771230D1EF4E6023123607A804A90556
:10281000AA06AB077F007E8C7D0A7C00121A81120B
:102820001B139068A1EEF0A3EFF0800A9068A174EA
:10283000FFF0A374B8F07E197F7D1230D1EF4E60A7
:102840000C12383DEF24D024FF92188002C2187E6B
:10285000197F831230D1EF4E60071236078F09803F
:1028600003E4F5097E197F891230D1EF4E600C1216
:10287000383DEF24D024FF92158002C2157E197FC7
:102880008F1230D1EF4E600C12383DEF24D024FF70
:1028900092108002C2107E197F951230D1EF4E60E7
:1028A0000C12383DEF24D024FF92138002C2137E15
:1028B000197F9B1230D1EF4E60071236078F0880C8
:1028C000037508407E197FA11230D1EF4E600712C8
:1028D00036078F0F8003750F057E197FA71230D141
:1028E000EF4E60071236078F0C8003E4F50C7F0073
:0128F00022C5
:1034C700C212C21AC214C211C217E4F510F50DF5E3
:1034D7000EF547C20FD297D296C219D216750BFFB7
:1034E7007511091227F0EF6003121C70C2ADE4F5E5
:1034F700C9D2CDD2CCC2C9C2CAF5CDF5CC9068A18C
:10350700E0F5CBA3E0F5CA85CBCD85CACCE4F59829
:1035170030100C2015095387BFD29FD29E8002D24C
:103527009E438740C29FC2ACC298C29975B81075B6
:09353700B710D2CAD29CD2AC221A
:0100220022BB
:102C6600E4FF0F2407F582E43461F583E511F00FE4
:102C760074072401F582E43461F583E4F07C667D13
:102C860094FEED1DAA0470011CF5828A83E0FBAA5E
:102C9600070F74072AF582E43461F583EBF00EBE64
:102CA60004E07C667D98E4FEED1DAA0470011CF527
:102CB600828A83E0FBAA070F74072AF582E434614F
:102CC600F583EBF00EBE04E07C667D9CE4FEED1D14
:102CD600AA0470011CF5828A83E0FBAA070F740719
:102CE6002AF582E43461F583EBF00EBE04E07C66DF
:102CF6007DA0E4FEED1DAA0470011CF5828A83E026
:102D0600FBAA070F74072AF582E43461F583EBF01A
:042D16000EBE04E009
:012D1A002296
:0A388F00C2992099FDD299D290222F
:09389900D2CAD29CD2ACC21422A6
:103540008F2630120B200A5B7E197FAD1229D722FD
:1035500090637BE0F511E52624FCFFF50D7D7C757D
:103560008363058263A2019067A163A20112219681
:10357000E4F510D212C296301804D20F800BE50980
:103580006004F544800312388F200A157E197FBB32
:103590001229D77E677FA1E52624FCFDE4FB122BD0
:0435A00092C21A2297
:102FAC00E50E547FFFD394005003023042E547D323
:102FBC00950F5009EFC395085003301979C219C207
:102FCC0091C2AF850E12630E80530E80E4F547C29A
:102FDC0011C214D2AF906478F0E512547FFFA3F0C5
:102FEC0090667CE090647AF0A3E511F0E5125480D1
:102FFC0024A1F582E43466F58363A20190647C63BA
:10300C00A201122196200A29309F077E197FC11236
:10301C0029D77E197FD01229D7E512548024A1F527
:10302C0082E43466AF82FEE512547FFDE4FB122B82
:09303C0092C29F7F01227F002255
:03001E00C2AC224F
:10377000300004C200050A300F08209705C20F125E
:10378000388FE544B40106E4F54412388F30120C4A
:10379000E50AD394144008C212D21A22E4F50A2290
:0B388400301A05C21A7F01227F0022CB
:10305100020881E493A3F8E493A34003F68001F20C
:1030610008DFF48029E493A3F85407240CC8C33380
:10307100C4540F4420C8834004F456800146F6DF4F
:10308100E4800B0102040810204080903805E47EA2
:10309100019360BCA3FF543F30E509541FFEE49344
:1030A100A360010ECF54C025E060A840B8E493A30B
:1030B100FAE493A3F8E493A3C8C582C8CAC583CA36
:1030C100F0A3C8C582C8CAC583CADFE9DEE780BEEE
:0138200000A7
:1019FF00BB010689828A83E0225002E722BBFE02E6
:091A0F00E32289828A83E4932218
:101A1800BB010CE58229F582E5833AF583E0225083
:101A280006E92582F8E622BBFE06E92582F8E222CD
:0D1A3800E58229F582E5833AF583E49322E7
:101A450075F008758200EF2FFFEE33FECD33CDCC58
:101A550033CCC58233C5829BED9AEC99E5829840DB
:101A65000CF582EE9BFEED9AFDEC99FC0FD5F0D6B8
:101A7500E4CEFBE4CDFAE4CCF9A88222B800C1B9E2
:101A85000059BA002DEC8BF084CFCECDFCE5F0CB20
:101A9500F97818EF2FFFEE33FEED33FDEC33FCEB59
:101AA50033FB10D703994004EB99FB0FD8E5E4F914
:101AB500FA227818EF2FFFEE33FEED33FDEC33FC01
:101AC500C933C910D7059BE99A4007EC9BFCE99AF5
:101AD500F90FD8E0E4C9FAE4CCFB2275F010EF2F3A
:101AE500FFEE33FEED33FDCC33CCC833C810D7073A
:101AF5009BEC9AE899400AED9BFDEC9AFCE899F875
:0E1B05000FD5F0DAE4CDFBE4CCFAE4C8F92207
:0E1B1300C3E49FFFE49EFEE49DFDE49CFC22E3
:101B2100EB9FF5F0EA9E42F0E99D42F0E89C45F01A
:011B31002291
:0C1B3200ECF0A3EDF0A3EEF0A3EFF02226
:101B3E00A8828583F0D083D082121B55121B5512BA
:101B4E001B55121B55E473E493A3C583C5F0C583DF
:101B5E00C8C582C8F0A3C583C5F0C583C8C582C8F1
:011B6E002254
:1013E800E53A242EF8E6053A22782B302202782EA8
:1013F800E475F001121BD00219FF201BEB7F2ED2DF
:101408001B8018EF540F2490D43440D4FF301F0BA6
:10141800EF24BFB41A0050032461FFE53B600215B6
:101428003B053EE53E7002053D30220D782BE47504
:10143800F001121BD0EF021B6F0236BD7403D222DB
:101448008003E4C222F53A8B2B8A2C892DE4F53BE4
:10145800F53DF53EE53B60077F2012142380F575C6
:101468003CFFC21CC21BC21DC21EC220C221C22315
:101478001213F1FF700D3022057F00121434AF3EB5
:10148800AE3D22B4255FC2D5C21F1213F1FF24D08E
:10149800B40A00501A75F00A783B30D50508B6FF33
:1014A8000106C6A426F620D5047002D21E80D924CF
:1014B800CFB41A00EF5004C2E5D21F021634D21C72
:1014C80080C6D21B80C0D21D80BCD2D580BAD220A3
:1014D80080B47F20121423201D077401B53B0040FF
:1014E800F11213E8FF12142302145CD223D22180D4
:1014F800951213E8FB1213E8FA1213E8F94A4B7035
:101508000679057A177BFF201D2EE53B602A7E00B1
:101518008E82758300121A1860060EEE653C70F014
:10152800C2D5EBC0E0EAC0E0E9C0E0EE12167BD01D
:10153800E0F9D0E0FAD0E0FB1219FFFF60AAEBC097
:10154800E0EAC0E0E9C0E0121423D0E02401F9D0B9
:10155800E03400FAD0E0FBE53C0460DCD53CD980FF
:10156800877BFF7A167977D21D809C791080027963
:1015780008C221C2238008D2D5790A8004790AC218
:10158800D5E53C047002F53CE4FAFDFEFF1213E8D1
:10159800FC7B08201C131213E8FD7B10301B0A1279
:1015A80013E8FE1213E8FF7B20EC3382D592D55066
:1015B80013C3E4301B069FFFE49EFEE4201C039D3A
:1015C800FDE49CFCE4CBF8C21CEC700CCFCECDCC77
:1015D800E824F8F870F38017C3EF33FFEE33FEED1D
:1015E80033FDEC33FCEB33FB994002FB0FD8E9EBFE
:1015F800301C05F8D0E0C448B21CC0E00AEC4D4EDF
:101608004F78207B0070C2EAB53C0040BCC0E012B5
:10161800167DD0F0D0E0201C04C4C0E0C4B21CC0C9
:10162800F012140CD0F0D5F0EB02145C121C2F143D
:10163800F95315735814CA4C14C64215774F157FC1
:0F16480044157F4914DF4315855515694615690B
:101657004515694717255014CE2D14D22E14F52B96
:1016670014D62314F320170E2A148E48000014ED05
:101677003F3F3F00790AA2D5201E14302009B91038
:10168700020404B9080104A2D52021025001042054
:101697001D68921DB53B005034C0E07F20301E19F5
:1016A7007F30A21D72217220500F1216D4C21DC2A4
:1016B70021C220C2237F30800F302003E9C0E0120F
:1016C7001423302003D0E0F9D0E0B53BCC3020170D
:1016D7007F30B9100C1214237F58301F077F788092
:1016E70003B90803121423301D057F2D0214237F2D
:1016F700202023F87F2B2021F322921D80CF286EF4
:10170700756C6C2900D21C1213E8301CF8C21C78C7
:101717003B30D50108F602148E2D50434958121359
:10172700E82403B405004001E49017209312141431
:0D173700743A121414D21E753B040215738F
:10226D008B2B8A2C892DE4F537F536F535F534F5BC
:10227D0032F533E52F4530452E6012EBC0E0EAC054
:10228D00E0E9C0E0AB2EAA2FA930121BE0AB2B0565
:10229D002DE52DAA2C7002052C14F91219FFF53815
:1022AD00C394094007E538D3940D40E1E538642027
:1022BD0060DBE538B42D054333038016E538B42BC8
:1022CD0005433301800C74FF252DF52D74FF352C3E
:1022DD00F52CE53160046410703FAB2BAA2CA92DB1
:1022ED001219FF64306009E531702E75310A8029AD
:1022FD00900001121A18FF64786004EFB45813436C
:10230D0033017531107402252DF52DE4352CF52C86
:10231D008007E5317003753108AB2B052DE52DAA2E
:10232D002C7002052C14F91219FFF538C394614075
:10233D000AE538D3947A50035338DF74D02538F535
:10234D0038C3940A400CE5389411406D74F9253862
:10235D00F538E538D39531506043330185373C85E9
:10236D00363B85353A853439AF317E00E4FCFDAB23
:10237D0037AA36A935A834121B81C8ECC8C9EDC9D6
:10238D00CAEECACBEFCBE4FCFDFEEB2538F537EEFC
:10239D003AF536ED39F535EC38F534AF37AE36ADB7
:1023AD0035FCAB3CAA3BA93AA839D3121B215003EB
:1023BD00022326433304022326E53320E003E48081
:1023CD002DE52F4530452E601EAB2BE52D24FFF955
:1023DD00E52C34FFFAEBC0E0EAC0E0E9C0E0AB2E3B
:1023ED00AA2FA930121BE0E53330E20774FFFFFE80
:1023FD00FDFC22E533AF37AE36AD35AC3430E103FD
:04240D00021B132279
:101B6F00BB010689828A83F0225002F722BBFE0155
:021B7F00F3224F
:101B8100E88FF0A4CC8BF0A42CFCE98EF0A42CFC03
:101B91008AF0EDA42CFCEA8EF0A4CDA8F08BF0A481
:101BA1002DCC3825F0FDE98FF0A42CCD35F0FCEBE0
:101BB1008EF0A4FEA9F0EB8FF0A4CFC5F02ECD39A5
:0F1BC100FEE43CFCEAA42DCE35F0FDE43CFC2212
:101BD000FAE6FB0808E6F925F0F618E6CA3AF62216
:101BE000BB011A89828A83D0F0D0E0F8D0E0F9D026
:101BF000E0FAD0E0FBE8C0E0C0F0021C5E5016E95D
:101C0000F8D083D082D0E0F9D0E0FAD0E0FBC082F7
:101C1000C083021C55BBFE16E9F8D083D082D0E009
:0F1C2000F9D0E0FAD0E0FBC082C083021C67223B
:101C2F00D083D082F8E4937012740193700DA3A344
:101C3F0093F8740193F5828883E473740293686058
:061C4F00EFA3A3A380DF58
:091C5500EBF608EAF608E9F622B4
:091C5E00EBF0A3EAF0A3E9F02287
:091C6700EBF208EAF208E9F222AE
:00000001FF
